:1000000000308A00A82E0000FF00030E8301A1002B
:100010000A08A0008A010408A2007708A300780853
:10002000A4007908A5007A08A6007B08A70083131E
:1000300083128C308400001D1F280C1938288D3045
:100040008400001C25280D183B2822088400230862
:10005000F7002408F8002508F9002608FA00270808
:10006000FB0020088A00210E8300FF0E7F0E09008E
:100070008A110A123E288A110A124B28941314136B
:1000800094121430AB00C3010730BB0094160C115E
:100090008A110A12252870147008831687008312AB
:1000A00007185428031055280314B00CAF0CB208DD
:1000B00003195C28B20390280314AF0DB00D03148C
:1000C000AF0DB00D0A30B2003408F700F70803197D
:1000D0007A280130770203197D280230770203194C
:1000E000802803307702031983280430770203192C
:1000F000862889283008BC008A283008BD008A2854
:100100003008BE008A283008BF008A283008C000A6
:100110008A288A28B40A33083402031D9028B517A8
:100120000D108A110A122528733084000008031963
:10013000A6280630F800F701F70B9C28F80B9B283F
:100140007B30F700F70BA228800B99288A110A123E
:10015000A52983160D1073088312B300B401F501AD
:10016000F010700883168700831287103130F70073
:10017000F70BB82800000000701070088316870085
:10018000831207103130F700F70BC428000000007D
:10019000F0147008831687008312F0147008831619
:1001A000870083128718CD28F4017408073C031CCC
:1001B00003297208F7007408F8000319E3280310F4
:1001C000F70CF80BDF28771CED28701470088316E5
:1001D00087000130F5068312F3287010700883162B
:1001E000870083120710F0147008831687008312AB
:1001F000871CF328F0147008831687008312871871
:10020000FA28F40AD528F0147008831687008312A0
:1002100087180329F508031D132970147008831625
:1002200087008312192970107008831687008312C3
:100230000710F0147008831687008312871C192991
:100240001030F700F70B2229000070147008831695
:1002500087008312F01470088316870083128718B2
:100260002A29F0147008831687008312871C31290D
:1002700070147008831687008312071C422901300E
:10028000F6004329F601F0147008831687008312E4
:10029000871843290D1083160D1483120034B51FDF
:1002A0004F29B501B40100343F3085008601FF308D
:1002B000870088018901203083168500FF30860081
:1002C0001F308700F000FF308800091089100911E5
:1002D000811383121F0838399F00063083169F0050
:1002E00083129412F012700883168700701670083B
:1002F00087008516F015700887003430831294004B
:10030000003083169400831207119701053097007F
:1003100087109D0104309D008530900083160D14D8
:10032000C03083128B04AE01FF30AF00FF30B0004D
:100330000A30B200B501B401C301A801A901AA01A4
:100340000230F200FA30F3009428F20BA229FF30B9
:10035000F2000330F300A9204F21FF30F2000330F8
:10036000F300A9204F21FF30F2000330F300A92051
:100370004F21F230F2000230F300A9204F21E93082
:10038000F2000330F300A9204F21F330F2000130D6
:10039000F300A9204F21C830F2000130F300A9205A
:1003A0004F21F330F2000130F300A9204F216430D7
:1003B000F2000130F300A9204F21F330F2000130A8
:1003C000F300A9204F215030F2000130F300A920A2
:1003D0004F21F230F2000230F300A9204F21F33018
:1003E000F2000130F300A9204F21C830F2000130A3
:1003F000F300A9204F21F330F2000130F300A920CF
:100400004F21C830F2000130F300A9204F21F33012
:10041000F2000130F300A9204F215030F2000130EA
:10042000F300A9204F21F230F2000230F300A9209E
:100430004F21F030F2000130F300A9204F21F430B9
:10044000F2000130F300A9204F211430AB00BB01B2
:1004500083160C1583128A110A12B22EEB30F200A9
:100460000530F300A9204F21FF30C100FF30C2004A
:1004700008086038C10006193E2A42118618412A30
:10048000C2113D1E4D2A3E08FF3C013EF10071089D
:10049000033C03184C2AC212522A3E08033C03189C
:1004A000522A4212BD1E5E2A3F08FF3C013EF10067
:1004B0007108073C03185D2AC213632A3F08073CF2
:1004C0000318632A4213BD1C662AC2103D1C692A08
:1004D0004210C01E6C2AC112401E6F2A4113881E92
:1004E000722AC112081F752A41133D1D7B2ABF3095
:1004F000C1000F30C20040080F39F100F1080319A4
:100500008C2AF11D882AFF30C1000B30C2008C2AD2
:10051000FF30C1000730C20083160D108312BB01EB
:100520008A110A12B72E000000000000000000002F
:10053000831605128312051200000000000000005F
:100540000000831605168312003470157008831698
:10055000870083120719A52A831614108312AB0192
:10056000FF30930094132B08033C031CFD2A8316D1
:100570001418BC2A8312B72A83121308AC009413F0
:1005800014132B08F700F7080319D32A0130770258
:100590000319D62A023077020319D92A03307702C9
:1005A0000319DC2AEB2A8230AD00EE2A5A30AD0066
:1005B000EE2A4108AD00EE2A4208AD004508C23CD3
:1005C000031DEA2A2C08803C031DEA2A0230A800F9
:1005D0001430AB00EE2A1430AD00EE2A2D08930043
:1005E00044302B0784002C0880005A302B078400ED
:1005F0002D0880009322AB0AB32A8A110A12CD2E4D
:10060000701570088316870083120719002B831654
:1006100014108312AB01FF30930094132B08073C96
:10062000031C782B83161418172B8312122B83129A
:100630001308AC00941314132B08F700F7080319E0
:100640003E2B013077020319492B02307702031940
:100650004C2B0330770203194F2B04307702031918
:10066000522B053077020319552B063077020319F8
:10067000582B0730770203195B2B662BCE30AD0069
:100680002C08803C0319482B1430AB000130C30008
:10069000692B5A30AD00692B4108AD00692B420827
:1006A000AD00692B0130AD00692B0130AD00692B25
:1006B0000130AD00692B0130AD004508C23C031D7F
:1006C000652B0230A8001430AB00692B1430AD004C
:1006D000692B2D08930044302B0784002C088000E0
:1006E0005A302B0784002D0880009322AB0A0E2B72
:1006F0008A110A12CF2E02302B02FA3E0318982BD1
:10070000063E9B2BC030AD00982B4030AD00982B9F
:10071000A908031D8D2BAD018F2B8030AD00982BC8
:100720004030AD00982B8030AD00982BAD01982B58
:100730008A110A12B62D0A148A140A118207822B12
:10074000852B882B902B932B962B02302B02FA3E75
:100750000318CD2B063ED02BAD01CD2BAD01CD2BFB
:100760008030AD00CD2BC708031DB92B4030AD0044
:10077000BB2B8030AD00CD2BC708031DC12BAD01B5
:10078000C32B8030AD00CD2BC708031DCA2B5030C2
:10079000AD00CC2B2830AD00CD2B8A110A12B82D1C
:1007A0000A148A140A118207AC2BAE2BB02BB32B80
:1007B000BC2BC42B02302B02FA3E0318EF2B063E53
:1007C000F22BAD01EF2BAD01EF2B4030AD00EF2B45
:1007D000AD01EF2B8030AD00EF2BAD01EF2B8A1177
:1007E0000A12BA2D0A148A140A118207E12BE32B8C
:1007F000E52BE82BEA2BED2B02302B02FA3E0318F7
:10080000162C063E192CAD01162CAD01162CAD018F
:10081000162CC708031D0F2C2030AD00112CE03022
:10082000AD00162CAD01162CAD01162C8A110A1242
:10083000BC2D0A108A100A158207032C052C072CE0
:10084000092C122C142C02302B02FA3E0318472CD0
:10085000063E552CAA08031D302CFF30AD00312C6C
:10086000AD01472CAA08031D382CFF30AD003A2CEF
:100870008030AD00472CFF30AD00472CFF30AD007D
:10088000472CFF30AD00472CFF30AD00472CC70888
:10089000031D512C4808803C031D512C0130AA0037
:1008A000522CAA018A110A12BE2D0A108A100A15AA
:1008B00082072A2C322C3B2C3E2C412C442CA9089C
:1008C000031D762C02302B02FA3E0318752C063ECF
:1008D000972CAD01752CAD01752CAD01752CAD01BA
:1008E000752CAD01752CAD01752C942C290B792C30
:1008F0007D2C2908023C031D942C02302B02FA3E69
:100900000318942C063EA12CFF30AD00942CFF3030
:10091000AD00942CC030AD00942CAD01942CAD01F1
:10092000942C5A30AD00942C8A110A12C02D0A1052
:100930008A100A158207692C6B2C6D2C6F2C712C78
:10094000732C0A108A100A158207842C872C8A2C93
:100950008D2C8F2C912C02302B02FA3E0318BE2CCA
:10096000063ED22CAD01BE2CAD01BE2CAD01BE2C7D
:10097000AD01BE2CAD01BE2CAD01BE2CC708031DC0
:10098000CF2C2908FD3E0318CF2C033EDC2CA801F8
:10099000CF2C0130A800CF2C0330A800CF2C8A1117
:1009A0000A12C22D0A108A100A158207B22CB42C22
:1009B000B62CB82CBA2CBC2C0A108A100A15820747
:1009C000C72CC92CCC2C02302B02FA3E0318F62C73
:1009D000063E042DAD01F62CAD01F62CAD01F62C32
:1009E000AD01F62CAD01F62CAD01F62C4708803C8C
:1009F000031DFD2C0130A900012DC708031D012D89
:100A0000A9018A110A12C42D0A148A100A15820734
:100A1000EA2CEC2CEE2CF02CF22CF42C02302B02D5
:100A2000FA3E0318222D063E272DAD01222DAD01E1
:100A3000222DAD01222DAD01222DAD01222D5A30E6
:100A4000AD00222D0230A9008A110A12C62D0A1407
:100A50008A100A158207152D172D192D1B2D1D2DF6
:100A60001F2D02302B02FA3E0318462D063E492D5B
:100A7000AD01462DAD01462D4030AD00462DAD01F6
:100A8000462DAD01462D5A30AD00462D8A110A1271
:100A9000C82D0A148A100A158207382D3A2D3C2DCC
:100AA0003F2D412D432D701570088316870083124A
:100AB0000719532D831614108312AB01FF309300D6
:100AC00094132B08073C031CDE2D831614186A2D83
:100AD0008312652D83121308AC0094131413AB0812
:100AE000031D7D2DCF30AD002C08803C03197C2DDB
:100AF0001430AB000130C300CF2D2B0B822D5A30A8
:100B0000AD00CF2D2B08013C0318CD2D2B08073C41
:100B1000031CCD2D4508F700A23077020319B52D2F
:100B2000623077020319B72DE23077020319B92D2D
:100B3000323077020319BB2DB23077020319BD2D75
:100B4000823077020319BF2DC23077020319C12DFD
:100B5000223077020319C32DF23077020319C52D15
:100B6000023077020319C72DC92D7B2BCC2DA52B65
:100B7000CC2DDA2BCC2DFC2BCC2D232CCC2D5F2C8B
:100B8000CC2DAB2CCC2DE32CCC2D0E2DCC2D312D02
:100B9000CC2D1430AD00CC2DCF2D1430AB002D0852
:100BA000930044302B0784002C0880005A302B0718
:100BB00084002D0880009322AB0A612D8A110A124D
:100BC000D12E701570088316870083120719E12D46
:100BD000831614108312AB01FF30930094132B087B
:100BE000133C031CA52E83161418F82D8312F32D25
:100BF00083121308AC00941314132B08F700F708A2
:100C000003194F2E0130770203195A2E0230770252
:100C100003195D2E033077020319602E043077022A
:100C20000319632E053077020319662E063077020A
:100C30000319692E0730770203196C2E08307702EA
:100C400003196F2E093077020319712E0A307702CB
:100C50000319732E0B3077020319752E0C307702AF
:100C60000319772E0D3077020319792E0E30770293
:100C700003197B2E0F30770203197D2E1030770277
:100C800003197F2E113077020319812E123077025B
:100C90000319832E133077020319852E932E9E306D
:100CA000AD002C08803C0319592E1430AB000130E4
:100CB000C300962E5A30AD00962E4208AD00962EF7
:100CC0004108AD00962E0130AD00962E0130AD00EA
:100CD000962E0130AD00962E0130AD00962EAD015E
:100CE000962EAD01962EAD01962EAD01962EAD013C
:100CF000962EAD01962EAD01962EAD01962EAD012C
:100D0000962EAD01962EAD01962EAD014508C23C42
:100D1000031D922E4708803C031D922E0230A8002E
:100D20001430AB00962E1430AD00962E2D08930093
:100D300044302B0784002C0880005A302B07840095
:100D40002D0880009322AB0AEF2D8A110A12D32EB0
:100D500084011F308305073083169F00FF30F000A9
:100D6000831254293B08073C031DB72E2E2AC308C3
:100D7000031DD52E2808F700F7080319CC2E0130E3
:100D800077020319CE2E023077020319D02E0330DA
:100D900077020319D22ED42EA52AD52E002BD52EBC
:0E0DA000532DD52EE12DD52ED52EB22E63006B
:02400E00723FFF
:00000001FF
